:020000040000FA
:040000000000C9280B
:080008002700931D1428931139
:1000100020003F1F0F28FF30A400A500A600BF1F2F
:100020001428B101B201B3012000911CB92891102C
:10003000B11B21283808B3073708B23D3608B13D57
:1000400027283B08B3073A08B23D3908B13D701183
:10005000031870150C1E36283C080B00B529BA2968
:10006000BF29C529CE29DD29EC29212A3C080B000E
:10007000252A312A402A482A582A682A782A952A85
:10008000701C4A282808A6072708A53D0030A43D73
:10009000031C51284608C800A9004708C900AA0047
:1000A00055282908C8002A08C9000E1A71284B08CB
:1000B000C9024A08C83B0308013A8300C80CC90CAE
:1000C000C837C90CC837C90CC837C90CC837C90CE0
:1000D0004908CB074808CA3D4B08CD004A08CC0068
:1000E00075284908CD004808CC00F401F5013D0809
:1000F00003104D1BF407F40CF50CCD1BF407F40CA6
:10010000F50C4C18F407F40CF50CCC18F407F40CAF
:10011000F50C4C19F407F40CF50CCC19F407F40C9D
:10012000F50C4C1AF407F40CF50CCC1AF407F40C8B
:10013000F50C4C1BF407F40CF50C0310CC1BF40766
:10014000F40CF50C03103D09CE00CF01CE36CF0CD8
:100150004F08F5074E08F43D2030F5070030F43D18
:1001600025009316F51F93121316751F13127408AA
:100170009100090021009D005030F100F10BBE28D4
:100180009D149D18C1281C08F0191C09F3002000BB
:1001900008002100F030990001309500FF308C00FC
:1001A000DF308E008B170B179114240030308C0039
:1001B00010308E0027000830910020009A01FF3097
:1001C0009B0000309C0025009E010C309300803085
:1001D0009100230007308C000F308E00210060302A
:1001E0009E00200085018701FF30BD008030BE00E9
:1001F000BC01FF30A600A500A400A701A801F001E2
:10020000BF015830AB00AC00AD00B301B201B10189
:10021000B401B501B601B701B801B901BA01BB011A
:10022000F201F0118C1EF0151C15F20A7208073944
:100230000B002129342940295D2961296D2978295C
:1002400015290130BA20840085018435850D0530DB
:1002500084078330853D400884070030853D1200C7
:10026000B4001200B50083290530BA20043E73069D
:10027000E039031D1529F30E73360739BC00152923
:100280000930BA20840085018435850D0530840746
:100290008330853D8A3084070030853D1200A700F9
:1002A0001200A800730870185929F839031D70143A
:1002B0001529FC390319701015291130BA20BD0019
:1002C00015291530BA20BE0014303E02031CBE02B0
:1002D000EB303E020318BE0283291930BA20043ED7
:1002E0007306C039031D15297308C039BF001529CD
:1002F0001D30BA20043E7306C039031D152973084A
:10030000C039C0001529A2010310340CA000350C1F
:10031000A100A20C3E08D4009E215008B60051084E
:10032000B7005208B8003E08003CD4009E21500897
:10033000B9005108BA005208BB001529D301183082
:10034000A3002008D0002108D1002208D200520DBD
:10035000D10DD00DD30DD20D5408D3020318521471
:10036000521CD307A30BA72908003108C600320886
:10037000C70040283109C6003209C7004028FF30B5
:10038000B11B0030C600C70040283235C700310D10
:10039000C600B11B4028C709C6094028310886009D
:1003A0003235860D870D8635870DF030860787300C
:1003B000873D3208C500DA224028310886003235F0
:1003C000860D870D8635870DF23086078B30873D89
:1003D0003208C500DA224028311B062A310886007F
:1003E00087013235860D0935860D0935860D870D55
:1003F0008635870DF43086078F30873D3208C5007B
:10040000DA22B11F4028C609C70940287F30C6003C
:10041000FF30C70040282C08B0002D08AF00AE0008
:100420002F0C300C2E06B00DAF0D2F08AE06B00D00
:100430002F0DAE062C08AD002B08AC002E08AB002B
:1004400008000B22C600C70140283108C600320848
:10045000C700C636C70C3208C70731087F39C63D0A
:100460004028C601C701B11B40283109C600320926
:10047000C700C735C60DC735C60DC735C60D4028E0
:10048000FF30B11B0030311A0030C600C7004028D1
:100490003108860087013235860D870D8635870D38
:1004A000F63086079330873D3208C500DA224028AF
:1004B0003108860087013235860D870D8635870D18
:1004C000F83086079730873D3208C500DA22402889
:1004D0003108860087013235860D870D8635870DF8
:1004E000FA3086079B30873D3208C500DA22402863
:1004F00032088600310887008736860C8736860CDE
:100500008736860C03308705FE308605F430860773
:100510008F30873D3208C500C535C535C535DA226F
:10052000B11F4028C609C7094028701D9B2A4308EF
:10053000C1000B22C300C601C7014108321B43089A
:10054000C607C60CC70C4108B21B4308C607C60C39
:10055000C70C410831184308C607C60CC70C410830
:10056000B1184308C607C60CC70C41083119430827
:10057000C607C60CC70C4108B1194308C607C60C0C
:10058000C70C4108311A4308C607C60CC70C4108FE
:10059000B11A4308C607C60CC70C4108311B4308F3
:1005A000C607C60CC70C4108B11B4308C607C60CDA
:1005B000C70C40281600C1001600C2001600C30078
:1005C0001600C4004108C6004208C7004208451A88
:1005D0004408C7074108451A4308C63DC60CC70C66
:1005E0004208C51A4408C7074108C51A4308C63D52
:1005F000C60CC70C4208451B4408C7074108451BE9
:100600004308C63DC60CC70C080000341B34003438
:100610001B3400341C3400341D3400341D340034C9
:100620001E3400341F3400341F34003420340034AE
:100630002134003421340034223400342334003493
:100640002434003424340034253400342634003477
:100650002734003428340034293400342934003459
:100660002A3400342B3400342C3400342D3400343C
:100670002E3400342F34003430340034313400341C
:1006800032340034333400343534003436340034FA
:100690003734003438340034393400343B340034D7
:1006A0003C3400343D3400343E34003440340034B3
:1006B000413400344334003444340034463400348C
:1006C00047340034493400344A3400344C34003464
:1006D0004E3400344F340034513400345334003439
:1006E0005534003456340034583400345A3400340D
:1006F0005C3400345E3400346034003462340034DE
:100700006534003467340034693400346B340034A9
:100710006E34003470340034733400347534003473
:10072000783400347A3400347D340034803400343A
:100730008234003485340034883400348B340034FF
:100740008E340034913400349534003498340034BD
:100750009B3400349F340034A2340034A634003477
:10076000A9340034AD340034B1340034B53400342D
:10077000B9340034BD340034C1340034C5340034DD
:10078000C9340034CE340034D2340034D734003489
:10079000DB340034E0340034E5340034EA3400342F
:1007A000EF340034F5340034FA340034FF340134CB
:1007B000053401340B34013411340134163401345E
:1007C0001D340134233401342934013430340134EC
:1007D000363401343D340134443401344B34013473
:1007E000523401345A3401346134013469340134EF
:1007F0007134013479340134813401348A34013460
:10080000923401349B340134A4340134AD340134C6
:10081000B7340134C1340134CA340134D43401341E
:10082000DF340134E9340134F4340134FF34023468
:100830000A34023415340234213402342D340234A3
:100840003934023446340234523402345F340234D0
:100850006D3402347A3402348834023496340234EB
:10086000A5340234B4340234C3340234D2340234F2
:10087000E2340234F23403340334033414340334E2
:100880002534033437340334493403345B340334BC
:100890006E3403348134033495340334A93403347F
:1008A000BD340334D2340334E8340334FE34043426
:1008B000143404342B340434423404345A340434AD
:1008C000723404348B340434A5340434BF34043417
:1008D000D9340434F5340534103405342D3405345A
:1008E0004A3405346734053486340534A534053478
:1008F000C4340534E534063406340634273406346B
:100900004A3406346D34063491340634B634063431
:10091000DC340734023407342934073451340734C3
:100920007B340734A4340734CF340734FB34083421
:10093000283408345534083484340834B434083442
:10094000E5340934173409344A3409347E3409341F
:10095000B3340934E9340A3421340A3459340A34BA
:1009600094340A34CF340B340B340B3449340B3405
:1009700089340B34C9340C340B340C344F340C34FC
:1009800094340C34DA340D3422340D346C340D3498
:10099000B7340E3404340E3453340E34A3340E34CE
:1009A000F5340F3449340F349F340F34F634103497
:1009B00050341034AB3411340834113468341134E9
:1009C000C93412342D34123493341234FB341334BA
:1009D00066341334D234143441341434B3341534FB
:1009E000273415349E3416341734163493341734A0
:1009F0001134173492341834173418349E3419349F
:100A000028341934B5341A3445341A34D8341B34E4
:100A10006E341C3408341C34A5341D3446341D3463
:100A2000EA341E3492341F343D341F34EC34203405
:100A30009F3421345634223411342234D0342334B8
:100A4000933424345A34253426342534F634263469
:100A5000CB342734A53428348334293466342A34FB
:100A60004E342B343B342C342E342D3425342E3458
:100A700022342F34253430342D3431343B34323465
:100A80004F3433346934343489343534B034363403
:100A9000DD343834103439344B343A348C343B340C
:100AA000D4343D3423343E347A343F34D834413462
:100AB0003E344234AC34443422344534A0344734D8
:100AC00026344834B5344A344C344B34ED344D3448
:100AD00096344F344934513406345234CC3454347F
:100AE0009C345634763458345B345A344A345C344B
:100AF00045345E344A3460345A3462347634643473
:100B00009E346634D234693413346B3460346D34BB
:100B1000BA347034213472349534753418347734DF
:100B2000A8347A3447347C34F4347F34B13482349A
:100B30007C3485345834883443348B343F348E3499
:100B40004C3491346934943499349734DA349B3486
:100B50002D349E349334A2340C34A5349834A93403
:100B60003834AC34ED34B034B634B4349534B834AD
:100B70008934BC349334C034B534C434ED34C9340E
:0A0B80003D34CD34A534D2342634C0
:100FE0008034003481349234833424348434B634ED
:100FF000863448348734D93489346A348A34FB34AB
:101000008C348C348E341C348F34AB3491343A3479
:101010009234C834943455349534E23497346E3471
:101020009834F9349A3482349C340B349D3493349C
:101030009F341A34A0349F34A2342334A334A6340A
:10104000A5342834A634A834A8342634A934A334CB
:10105000AB341F34AC349934AE341134AF348734EC
:10106000B034FB34B2346E34B334DF34B5344D3481
:10107000B634BA34B8342434B9348C34BA34F23493
:10108000BC345634BD34B834BF341734C034733430
:10109000C134CE34C3342534C4347A34C534CD3469
:1010A000C7341C34C8346934C934B434CA34FB344A
:1010B000CC343F34CD348134CE34BF34CF34FB34E0
:1010C000D1343334D2346834D3349B34D434C93437
:1010D000D534F534D7341D34D8344234D93464345B
:1010E000DA348234DB349C34DC34B334DD34C7345A
:1010F000DE34D734DF34E334E034EB34E134F0343D
:10110000E234F134E334EE34E434E834E534DD340D
:10111000E634CF34E734BC34E834A634E9348B34D5
:10112000EA346D34EB344A34EC342334EC34F834A0
:10113000ED34C934EE349634EF345E34F034223476
:10114000F034E234F1349D34F2345434F33407345F
:10115000F334B534F4345F34F5340434F534A53461
:10116000F6344134F634D834F7346B34F734FA3487
:10117000F8348434F9340934F9348934FA340534D0
:10118000FA347C34FA34EE34FB345C34FB34C5344A
:10119000FC342934FC348834FC34E334FD343934F1
:1011A000FD348934FD34D534FE341D34FE345F34CF
:1011B000FE349C34FE34D534FF340934FF343734E4
:1011C000FF346134FF348634FF34A634FF34C13435
:1011D000FF34D834FF34E934FF34F534FF34FD34C0
:1011E000FF34FF34FF34FD34FF34F534FF34E93489
:1011F000FF34D834FF34C134FF34A634FF3486348E
:10120000FF346134FF343734FF340934FE34D534CD
:10121000FE349C34FE345F34FE341D34FD34D5344A
:10122000FD348934FD343934FC34E334FC348834FF
:10123000FC342934FB34C534FB345C34FA34EE34EA
:10124000FA347C34FA340534F9348934F934093405
:10125000F8348434F734FA34F7346B34F634D83451
:10126000F6344134F534A534F5340434F4345F34C1
:10127000F334B534F3340734F2345434F1349D3458
:10128000F034E234F0342234EF345E34EE34963409
:10129000ED34C934EC34F834EC342334EB344A34D0
:1012A000EA346D34E9348B34E834A634E734BC34A2
:1012B000E634CF34E534DD34E434E834E334EE347A
:1012C000E234F134E134F034E034EB34DF34E3344D
:1012D000DE34D734DD34C734DC34B334DB349C340F
:1012E000DA348234D9346434D8344234D7341D34B7
:1012F000D534F534D434C934D3349B34D23468343F
:10130000D1343334CF34FB34CE34BF34CD34813494
:10131000CC343F34CA34FB34C934B434C8346934AF
:10132000C7341C34C534CD34C4347A34C334253482
:10133000C134CE34C0347334BF341734BD34B83400
:10134000BC345634BA34F234B9348C34B83424341E
:10135000B634BA34B5344D34B334DF34B2346E34C9
:10136000B034FB34AF348734AE341134AC349934F8
:10137000AB341F34A934A334A8342634A634A8349B
:10138000A5342834A334A634A2342334A0349F34A3
:101390009F341A349D3493349C340B349A34823401
:1013A0009834F93497346E349534E23494345534A7
:1013B0009234C83491343A348F34AB348E341C3484
:1013C0008C348C348A34FB3489346A348734D9348D
:1013D000863448348434B6348334243481349234AB
:1013E000803400347E346E347C34DC347B344A34D4
:1013F0007934B834783427347634963475340534F7
:10140000733474347134E434703455346E34C63407
:101410006D3438346B34AB346A341E3468349234EF
:101420006734073465347E346334F53462346D34A4
:101430006034E6345F3461345D34DD345C345A3416
:101440005A34D834593458345734DA3456345D3435
:101450005434E134533467345134EF3450347934F4
:101460004F3405344D3492344C3421344A34B3343F
:10147000493446344734DC344634743445340E340D
:101480004334AA34423448344034E9343F348D3450
:101490003E3432343C34DB343B3486343A343334F7
:1014A0003834E4343734973436344C3435340534F6
:1014B0003334C13432347F34313441343034053440
:1014C0002E34CD342D3498342C3465342B343734C9
:1014D0002A340B342834E3342734BE3426349C3485
:1014E00025347E342434643423344D342234393466
:1014F0002134293420341D341F3415341E34103463
:101500001D340F341C3412341B3418341A34233471
:10151000193431341834443417345A341634753489
:10152000153493341434B6341334DD34133408349E
:101530001234373411346A341034A2340F34DE34A8
:101540000F341E340E3463340D34AC340C34F9349F
:101550000C344B340B34A1340A34FC340A345B347D
:101560000934BF3409342834083495340834063437
:1015700007347C340634F734063477340534FB34CE
:1015800005348434053412340434A43404343B3434
:101590000334D7340334783403341D340234C7346D
:1015A0000234773402342B340134E3340134A1346F
:1015B0000134643401342B340034F7340034C9343A
:1015C00000349F3400347A3400345A3400343F34C9
:1015D000003428340034173400340B34003403341E
:1015E000003401340034033400340B340034173435
:1015F0000034283400343F3400345A3400347A3410
:1016000000349F340034C9340034F73401342B34AF
:10161000013464340134A1340134E33402342B3412
:10162000023477340234C73403341D34033478343D
:101630000334D73404343B340434A4340534123432
:10164000053484340534FB34063477340634F734F7
:1016500007347C340834063408349534093428348B
:101660000934BF340A345B340A34FC340B34A134FB
:101670000C344B340C34F9340D34AC340E34633444
:101680000F341E340F34DE341034A23411346A3473
:1016900012343734133408341334DD341434B6348C
:1016A000153493341634753417345A34183444349A
:1016B000193431341A3423341B3418341C341234A2
:1016C0001D340F341E3410341F34153420341D34AF
:1016D000213429342234393423344D3424346434CD
:1016E00025347E3426349C342734BE342834E33405
:1016F0002A340B342B3437342C3465342D3498345D
:101700002E34CD34303405343134413432347F34E6
:101710003334C1343534053436344C3437349734AB
:101720003834E4343A3433343B3486343C34DB34B8
:101730003E3432343F348D344034E934423448341A
:101740004334AA3445340E34463474344734DC34DC
:10175000493446344A34B3344C3421344D34923411
:101760004F340534503479345134EF3453346734C2
:101770005434E13456345D345734DA3459345834FF
:101780005A34D8345C345A345D34DD345F346134D7
:101790006034E63462346D346334F53465347E3459
:1017A00067340734683492346A341E346B34AB3493
:1017B0006D3438346E34C634703455347134E43496
:1017C000733474347534053476349634783427346D
:1017D0007934B8347B344A347C34DC347E346E342F
:1017E00080340034FF34FF34FE346D34FC34DB3499
:1017F000FB344934F934B734F8342534F6349334AF
:10180000F5340134F3346F34F134DE34F0344C34D5
:10181000EE34BB34ED342A34EB349934EA340834F2
:10182000E8347834E634E734E5345734E334C83404
:10183000E2343834E034A934DF341A34DD348B3404
:10184000DB34FD34DA346F34D834E134D7345434F3
:10185000D534C734D4343B34D234AF34D1342334C8
:10186000CF349834CE340E34CC348434CA34FA3481
:10187000C9347134C734E834C6346034C434D9341C
:10188000C3345234C134CB34C0344634BE34C03493
:10189000BD343C34BB34B834BA343534B834B234E3
:1018A000B7343034B534AF34B4342F34B234AF3409
:1018B000B1343034AF34B234AE343434AC34B83400
:1018C000AB343C34A934C134A8344734A634CD34C5
:1018D000A5345534A334DD34A2346734A034F13454
:1018E0009F347C349E3408349C3495349B342334A8
:1018F0009934B234983442349634D23495346434C2
:101900009334F73492348B34913420348F34B6349A
:101910008E344D348C34E6348B347F348A341A342C
:101920008834B534873452348534F03484348F3479
:1019300083342F348134D134803474347F34183478
:101940007D34BD347C3463347B340B347934B4342B
:1019500078345E3477340A347534B734743465348B
:10196000733415347134C634703478346F342C3495
:101970006D34E1346C3497346B344F346A34093449
:101980006834C4346734803466343E346434FD349F
:101990006334BE3462348034613444346034093496
:1019A0005E34D0345D3498345C3462345B342D342E
:1019B0005934FB345834C93457349A3456346C345F
:1019C00055343F34543414345234EB345134C43429
:1019D00050349E344F347A344E3458344D34373486
:1019E0004C3418344A34FB344934DF344834C63478
:1019F0004734AE34463497344534833444347134F8
:101A00004334603442345134413444344034383403
:101A10003F342F343E3427343D3422343C341E349A
:101A20003B341C343A341C3439341E3438342134B9
:101A30003734273436342F3435343834343444345E
:101A40003334513432346134313472343034863486
:101A50002F349B342E34B3342D34CC342C34E8342E
:101A60002C3405342B3425342A34463429346A3452
:101A7000283490342734B8342634E13426340D34F5
:101A800025343C3424346C3423349E342234D3340F
:101A9000223409342134423420347D341F34BA34A2
:101AA0001E34F9341E343A341D347E341C34C434AC
:101AB0001C340B341B3456341A34A2341934F03429
:101AC00019344134183494341734E9341734413418
:101AD00016349A341534F634153454341434B53479
:101AE0001434183413347D341234E43412344D3445
:101AF0001134B934113427341034983410340A3482
:101B00000F3480340E34F7340E3471340D34ED3428
:101B10000D346B340C34EC340C346F340B34F4343B
:101B20000B347C340B3406340A3492340A342134B6
:101B30000934B234093446340834DC34083474349B
:101B400008340F340734AC3407344B340634ED34E6
:101B500006349234063438340534E13405348D3497
:101B600005343B340434EB3404349E3404345334AD
:101B700004340B340334C534033481340334403427
:101B8000033402340234C53402348C340234543405
:101B900002341F340134ED340134BD3401348F3448
:101BA0000134643401343C34013415340034F234EB
:101BB0000034D0340034B2340034953400347B34F3
:101BC0000034643400344F3400343C3400342C345A
:101BD00000341F340034143400340B340034053422
:101BE000003401340034003400340134003405344E
:101BF00000340B340034143400341F3400342C34DB
:101C000000343C3400344F340034643400347B34CA
:101C1000003495340034B2340034D0340034F2341B
:101C20000134153401343C340134643401348F34CC
:101C30000134BD340134ED3402341F3402345434E1
:101C400002348C340234C534033402340334403457
:101C5000033481340334C53404340B340434533432
:101C600004349E340434EB3405343B3405348D3471
:101C70000534E13406343834063492340634ED3415
:101C800007344B340734AC3408340F34083474341C
:101C90000834DC34093446340934B2340A3421348B
:101CA0000A3492340B3406340B347C340B34F43461
:101CB0000C346F340C34EC340D346B340D34ED349F
:101CC0000E3471340E34F7340F34803410340A3447
:101CD00010349834113427341134B93412344D345B
:101CE0001234E43413347D34143418341434B534D9
:101CF000153454341534F63416349A3417344134C8
:101D00001734E93418349434193441341934F03424
:101D10001A34A2341B3456341C340B341C34C434EF
:101D20001D347E341E343A341E34F9341F34BA3430
:101D300020347D3421344234223409342234D334E3
:101D400023349E3424346C3425343C3426340D340E
:101D50002634E1342734B8342834903429346A34B2
:101D60002A3446342B3425342C3405342C34E834CE
:101D70002D34CC342E34B3342F349B343034863469
:101D80003134723432346134333451343434443481
:101D90003534383436342F3437342734383421341A
:101DA00039341E343A341C343B341C343C341E3435
:101DB0003D3422343E3427343F342F3440343834D9
:101DC0004134443442345134433460344434713403
:101DD00045348334463497344734AE344834C634BB
:101DE0004934DF344A34FB344C3418344D343734FE
:101DF0004E3458344F347A3450349E345134C434D1
:101E00005234EB345434143455343F3456346C3437
:101E100057349A345834C9345934FB345B342D3434
:101E20005C3462345D3498345E34D03460340934C8
:101E300061344434623480346334BE346434FD34F9
:101E400066343E34673480346834C4346A340934C8
:101E50006B344F346C3497346D34E1346F342C343C
:101E6000703478347134C634733415347434653452
:101E70007534B73477340A3478345E347934B43412
:101E80007B340B347C3463347D34BD347F3418347C
:101E9000803474348134D13483342F3484348F3497
:101EA0008534F034873452348834B5348A341A3463
:101EB0008B347F348C34E6348E344D348F34B634E6
:101EC0009134203492348B349334F7349534643421
:101ED0009634D234983442349934B2349B34233417
:101EE0009C3495349E3408349F347C34A034F134CF
:101EF000A2346734A334DD34A5345534A634CD344C
:101F0000A8344734A934C134AB343C34AC34B8348D
:101F1000AE343434AF34B234B1343034B234AF349C
:101F2000B4342F34B534AF34B7343034B834B23479
:101F3000BA343534BB34B834BD343C34BE34C03428
:101F4000C0344634C134CB34C3345234C434D934AD
:101F5000C6346034C734E834C9347134CA34FA340E
:101F6000CC348434CE340E34CF349834D13423344A
:101F7000D234AF34D4343B34D534C734D73454346A
:101F8000D834E134DA346F34DB34FD34DD348B346F
:101F9000DF341A34E034A934E2343834E334C8345A
:101FA000E5345734E634E734E8347834EA34083436
:101FB000EB349934ED342A34EE34BB34F0344C3401
:101FC000F134DE34F3346F34F5340134F6349334C1
:101FD000F8342534F934B734FB344934FC34DB3479
:101FE000FE346D34FF34FF347F34FF3480340034EA
:101FF00080340134803405348034093480340E3424
:102000008034153480341D348034263480343134A7
:1020100080343D3480344A348034583480346734DA
:102020008034783480348A3480349D348034B134C0
:102030008034C7348034DD348034F53481340F3457
:10204000813429348134453481346234813480349C
:1020500081349F348134C0348134E1348234043497
:102060008234293482344E348234753482349C3440
:102070008234C5348234F03483341B34833448349E
:10208000833476348334A5348334D53484340634AD
:102090008434393484346D348434A2348434D83470
:1020A0008534103485344834853482348534BD34E5
:1020B0008534F93486343634863475348634B53410
:1020C0008634F5348734373487347A348734BF34F0
:1020D0008834043488344B34883493348834DC3482
:1020E00089342634893471348934BD348A340B34CC
:1020F0008A3459348A34A9348A34FA348B344C34CF
:102100008B349F348B34F4348C3449348C34A03485
:102110008C34F7348D3450348D34AA348E340534F5
:102120008E3461348E34BE348F341C348F347C341E
:102130008F34DC3490343D349034A0349134043402
:10214000913468349134CE349234353492349D34A1
:1021500093340634933470349334DB3494344734FA
:102160009434B43495342234953491349634023412
:10217000963473349634E534973458349734CD34E8
:10218000983442349834B83499342F349934A8347C
:102190009A3421349A349B349B3416349B349334D0
:1021A0009C3410349C348E349D340D349D348D34E5
:1021B0009E340E349E3490349F3413349F349734BD
:1021C000A0341B34A034A134A1342834A134AF345A
:1021D000A2343734A234C134A3344B34A334D634BC
:1021E000A4346234A434EF34A5347D34A6340B34E3
:1021F000A6349B34A7342B34A734BC34A8344E34D3
:10220000A834E134A9347534AA340934AA349F348B
:10221000AB343534AB34CC34AC346434AC34FC340F
:10222000AD349634AE343034AE34CB34AF3467345E
:10223000B0340434B034A134B1343F34B134DE347A
:10224000B2347E34B3341E34B334BF34B434613466
:10225000B5340434B534A734B6344B34B634F03422
:10226000B7349534B8343B34B834E234B9348A34B2
:10227000BA343234BA34DB34BB348434BC342E3414
:10228000BC34D934BD348534BE343134BE34DE344C
:10229000BF348B34C0343934C034E834C13497345B
:1022A000C2344734C234F734C334A834C4345A3443
:1022B000C5340C34C534BF34C6347234C734263404
:1022C000C734DA34C8348F34C9344534C934FB34A4
:1022D000CA34B134CB346834CC342034CC34D83420
:1022E000CD349134CE344A34CF340334CF34BD347A
:1022F000D0347834D1343334D134EE34D234AA34B7
:10230000D3346634D4342334D434E034D5349D34D7
:10231000D6345B34D7341A34D734D834D8349734DD
:10232000D9345734DA341734DA34D734DB349834C8
:10233000DC345834DD341A34DD34DB34DE349D349F
:10234000DF346034E0342234E034E534E134A8345E
:10235000E2346C34E3342F34E334F334E434B8340B
:10236000E5347C34E6344134E7340634E734CC34A5
:10237000E8349134E9345734EA341D34EA34E33430
:10238000EB34AA34EC347034ED343734ED34FE34AD
:10239000EE34C534EF348C34F0345434F1341B341F
:1023A000F134E334F234AB34F3347334F4343B3487
:1023B000F5340434F534CC34F6349434F7345D34E5
:1023C000F8342634F834EE34F934B734FA3480343F
:1023D000FB344934FC341234FC34DB34FD34A43493
:1023E000FE346D34FF343634FF34FF34FF3436347A
:1023F000FE346D34FD34A434FC34DB34FC3412344C
:10240000FB344934FA348034F934B734F834EE34D8
:10241000F8342634F7345D34F6349434F534CC345F
:10242000F5340434F4343B34F3347334F234AB34E1
:10243000F134E334F1341B34F0345434EF348C345D
:10244000EE34C534ED34FE34ED343734EC347034CE
:10245000EB34AA34EA34E334EA341D34E934573433
:10246000E8349134E734CC34E7340634E63441348C
:10247000E5347C34E434B834E334F334E3342F34D7
:10248000E2346C34E134A834E034E534E03422340E
:10249000DF346034DE349D34DD34DB34DD341A3433
:1024A000DC345834DB349834DA34D734DA34173443
:1024B000D9345734D8349734D734D834D7341A343D
:1024C000D6345B34D5349D34D434E034D43423341E
:1024D000D3346634D234AA34D134EE34D1343334E4
:1024E000D0347834CF34BD34CF340334CE344A348E
:1024F000CD349134CC34D834CC342034CB3468341B
:10250000CA34B134C934FB34C9344534C8348F3487
:10251000C734DA34C7342634C6347234C534BF34D1
:10252000C5340C34C4345A34C334A834C234F734F8
:10253000C2344734C1349734C034E834C0343934F9
:10254000BF348B34BE34DE34BE343134BD348534D4
:10255000BC34D934BC342E34BB348434BA34DB3488
:10256000BA343234B9348A34B834E234B8343B340F
:10257000B7349534B634F034B6344B34B534A7346C
:10258000B5340434B4346134B334BF34B3341E349A
:10259000B2347E34B134DE34B1343F34B034A1349B
:1025A000B0340434AF346734AE34CB34AE3430346A
:1025B000AD349634AC34FC34AC346434AB34CC3409
:1025C000AB343534AA349F34AA340934A934753471
:1025D000A834E134A8344E34A734BC34A7342B34A7
:1025E000A6349B34A6340B34A5347D34A434EF34A4
:1025F000A4346234A334D634A3344B34A234C1346B
:10260000A2343734A134AF34A1342834A034A134F7
:10261000A0341B349F3497349F3413349E34903449
:102620009E340E349D348D349D340D349C348E3460
:102630009C3410349B3493349B3416349A349B343A
:102640009A3421349934A83499342F349834B834D6
:10265000983442349734CD34973458349634E53432
:10266000963473349634023495349134953422344C
:102670009434B434943447349334DB349334703426
:102680009334063492349D34923435349134CE34BC
:1026900091346834913404349034A03490343D340F
:1026A0008F34DC348F347C348F341C348E34BE341D
:1026B0008E3461348E3405348D34AA348D345034E4
:1026C0008C34F7348C34A0348C3449348B34F43467
:1026D0008B349F348B344C348A34FA348A34A934A2
:1026E0008A3459348A340B348934BD348934713492
:1026F000893426348834DC348834933488344B3439
:10270000883404348734BF3487347A348734373498
:102710008634F5348634B5348634753486343634AC
:102720008534F9348534BD34853482348534483475
:10273000853410348434D8348434A23484346D34F1
:1027400084343934843406348334D5348334A53422
:10275000833476348334483483341B348234F03405
:102760008234C53482349C348234753482344E349D
:1027700082342934823404348134E1348134C034E5
:1027800081349F34813480348134623481344534DF
:102790008134293481340F348034F5348034DD348D
:1027A0008034C7348034B13480349D3480348A34EA
:1027B00080347834803467348034583480344A34F8
:1027C00080343D34803431348034263480341D34B8
:1027D0008034153480340E34803409348034053428
:1027E00080340134803400347F34FF34803400344A
:1027F0008234CD3485349934883464348B342F3426
:102800008D34F8349034BF3493348534963448345E
:10281000993408349B34C4349E347E34A134333428
:10282000A334E534A6349234A9343A34AB34DD34DD
:10283000AE347B34B1341234B334A434B6342F34D0
:10284000B834B434BB343134BD34A734C034153457
:10285000C2347B34C434DA34C7342F34C9347C34C2
:10286000CB34BF34CD34FA34D0342A34D23451345A
:10287000D4346D34D6347F34D8348734DA34833466
:10288000DC347534DE345B34E0343534E234043423
:10289000E334C634E5347D34E7342734E834C434D3
:1028A000EA345534EB34D834ED344F34EE34B834A4
:1028B000F0341434F1346334F234A334F334D634C2
:1028C000F434FB34F6341234F7341B34F834153452
:1028D000F9340234F934DF34FA34AF34FB346F3472
:1028E000FC342134FC34C534FD345A34FD34E03436
:1028F000FE345734FE34C034FF341934FF346434AA
:10290000FF34A134FF34CE34FF34ED34FF34FD34D2
:10291000FF34FF34FF34F234FF34D634FF34AC34A8
:10292000FF347334FF342D34FE34D834FE34743421
:10293000FE340334FD348434FC34F734FC345D3429
:10294000FB34B534FB340034FA343D34F9346D349F
:10295000F8349134F734A734F634B134F534AF3465
:10296000F434A134F3348634F2346034F1342E3448
:10297000EF34F134EE34A934ED345634EB34F8341A
:10298000EA348F34E9341D34E734A034E6341A34A1
:10299000E4348B34E234F234E1345034DF34A6349E
:1029A000DD34F334DC343934DA347634D834AC34CE
:1029B000D634DB34D5340334D3342434D1343F34E7
:1029C000CF345434CD346334CB346D34C9347234A1
:1029D000C7347234C5346E34C3346534C1345934A9
:1029E000BF344934BD343634BB342034B9340834B0
:1029F000B634ED34B434D134B234B334B034943466
:102A0000AE347434AC345334AA343234A834113470
:102A1000A534F134A334D134A134B2349F34953485
:102A20009D3479349B345F3499344834973433344B
:102A30009534213493341234913406348E34FF3477
:102A40008C34FB348A34FC348934023487340C34BB
:102A500085341C348334313481344C347F346D34C8
:102A60007D3495347B34C3347934F734783433345B
:102A7000763476347434C1347334133471346D3431
:102A80006F34D0346E343B346C34AE346B342B340E
:102A90006934B03468343F346634D73465347934BB
:102AA000643424346234D934613499346034623407
:102AB0005F3436345E3415345C34FE345B34F234C7
:102AC0005A34F1345934FA3459340F3458342F34D9
:102AD00057345A34563490345534D23455341F3424
:102AE000543478345334DC3453344C345234C83492
:102AF00052344F345134E2345134803451342A3416
:102B00005034E0345034A13450346E3450344734AF
:102B100050342B3450341B345034163450341C345D
:102B200050342E3450344B34503473345034A63433
:102B30005034E53451342E34513481345134E0343E
:102B4000523449345234BC3453343A345334C1349B
:102B5000543453345434EE3455349334563441346D
:102B60005634F9345734BA345834833459345634DB
:102B70005A3430345B3413345B34FE345C34F13417
:102B80005D34EC345E34EE345F34F7346134073452
:102B900062341E3463343B3464345F3465348834C7
:102BA0006634B7346734EB34693425346A346434BA
:102BB0006B34A7346C34EE346E343A346F34893469
:102BC0007034DC347234323473348B347434E7341C
:102BD000763445347734A534793406347A346A341B
:102BE0007B34CE347D3434347E349A3480340034B3
:102BF000813466348234CC3484343234853496342F
:102C00008634FA3488345B348934BB348B341934D9
:102C10008C3475348D34CE348F34243490347734FE
:102C20009134C634933412349434593495349C34EA
:102C30009634DB3498341534993449349A347834E2
:102C40009B34A1349C34C5349D34E2349E34F93431
:102C5000A0340934A1341234A2341434A3340F3410
:102C6000A4340234A434ED34A534D034A634AA34C8
:102C7000A7347D34A8344634A9340734A934BF348A
:102C8000AA346D34AB341234AB34AD34AC343F348D
:102C9000AC34C634AD344434AD34B734AE342034FF
:102CA000AE347F34AE34D234AF341B34AF345A3404
:102CB000AF348D34AF34B534AF34D234AF34E434C0
:102CC000AF34EA34AF34E534AF34D534AF34B9344B
:102CD000AF349234AF345F34AF342034AE34D634B2
:102CE000AE348034AE341E34AD34B134AD34383407
:102CF000AC34B434AC342434AB348834AA34E13446
:102D0000AA342E34A9347034A834A634A734D1346C
:102D1000A634F134A6340634A5340F34A4340E346A
:102D2000A3340234A134EB34A034CA349F349E342B
:102D30009E3467349D3427349B34DC349A34873492
:102D4000993429349734C134963450349434D5347A
:102D5000933452349134C534903430348E349334B7
:102D60008C34ED348B343F3489348A348734CD3419
:102D70008634093484343D3482346B348034933463
:102D80007E34B4347C34CF347A34E4347834F4345C
:102D90007634FE34753404347334053471340134BC
:102DA0006E34FA346C34EE346A34DF346834CD3443
:102DB0006634B8346434A1346234873460346B349C
:102DC0005E344E345C342F345A340F345734EF347D
:102DD0005534CE345334AD3451348C344F346C3498
:102DE0004D344D344B342F34493413344634F83495
:102DF0004434E0344234CA344034B7343E34A73427
:102E00003C349B343A34923438348E3436348E34F5
:102E10003434933432349D343034AC342E34C134B1
:102E20002C34DC342A34FD3429342534273454340A
:102E300025348A342334C73422340D3420345A34B0
:102E40001E34B0341D340E341B3475341934E6345A
:102E5000183460341634E3341534713414340834BF
:102E60001234AA341134573410340F340E34D2349F
:102E70000D34A0340C347A340B345F340A345134BA
:102E800009344F340834593407346F3406349334DA
:102E90000534C3340534003404344B340334A334D0
:102EA0000334093402347C340134FD3401348C346D
:102EB000013428340034D33400348D340034543495
:102EC00000342A3400340E34003401340034033426
:102ED000003413340034323400345F3400349C3412
:102EE0000034E734013440340134A934023420344E
:102EF0000234A63403343B340334DF3404349134D5
:102F000005345134063421340634FE340734EB34AE
:102F10000834E5340934EE340B3405340C342A34E7
:102F20000D345D340E349D340F34EC341134483498
:102F30001234B134143428341534AB3417343C34DF
:102F40001834D9341A3483341C343A341D34FC34E4
:102F50001F34CB342134A53423348B3425347D34D1
:102F600027347934293481342B3493342D34AF34DD
:102F70002F34D63432340634343441343634843445
:102F80003834D1343B3426343D3485343F34EB344B
:102F9000423459344434CF3447344C344934D13436
:102FA0004C345C344E34EE34513485345434233450
:102FB0005634C63459346E345C341B345E34CD34EC
:102FC0006134823464343C346634F8346934B8345F
:102FD0006C347B346F344134723408347434D134FB
:102FE00077349C347A3467347D343334803400341D
:102FF000803400348334C73487348D348B34523476
:103000008F3413349234D23496348B349A3440341F
:103010009D34EE34A1349534A5343434A834CB3403
:10302000AC345734AF34DA34B3345134B634BC34FE
:10303000BA341B34BD346C34C034AE34C334E234DF
:10304000C7340634CA341934CD341C34D0340D346A
:10305000D234EB34D534B634D8346E34DB34123455
:10306000DD34A234E0341C34E2348134E434D0342E
:10307000E7340834E9342A34EB343434ED3427347B
:10308000EF340234F034C634F2347134F43403349F
:10309000F5347D34F634DF34F8342734F9345634DB
:1030A000FA346D34FB346A34FC344E34FD34193454
:1030B000FD34CC34FE346534FE34E634FF344E3413
:1030C000FF349E34FF34D634FF34F734FF34FF34FA
:1030D000FF34F134FF34CB34FF348F34FF343D34CC
:1030E000FE34D534FE345834FD34C734FD34213435
:1030F000FC346734FB349A34FA34BB34F934C934C1
:10310000F834C634F734B234F6348E34F5345B34E4
:10311000F4341934F234C934F1346B34F0340134FA
:10312000EE348B34ED340A34EB347F34E934EA3452
:10313000E8344C34E634A634E434F934E334463429
:10314000E1348D34DF34CF34DE340E34DC344934B2
:10315000DA348234D834B934D634F034D534273420
:10316000D3345F34D1349834CF34D434CE3414349F
:10317000CC345734CA349F34C834ED34C734413466
:10318000C5349D34C4340034C2346B34C034E034AC
:10319000BF345E34BD34E734BC347B34BB341B34C1
:1031A000B934C734B8348034B7344634B6341B34F9
:1031B000B434FD34B334EF34B234EF34B2340034C9
:1031C000B1342034B0345234AF349434AE34E734B4
:1031D000AE344B34AD34C234AD344A34AC34E43460
:1031E000AC349034AC344F34AC342134AC3405348A
:1031F000AB34FC34AC340534AC342134AC344F340F
:10320000AC349034AC34E434AD344A34AD34C234EC
:10321000AE344B34AE34E734AF349434B03452343B
:10322000B1342034B2340034B234EF34B334EF3438
:10323000B434FD34B6341B34B7344634B834803437
:10324000B934C734BB341B34BC347B34BD34E734AD
:10325000BF345E34C034E034C2346B34C434003420
:10326000C5349D34C7344134C834ED34CA349F3436
:10327000CC345734CE341434CF34D434D13498349D
:10328000D3345F34D5342734D634F034D834B93419
:10329000DA348234DC344934DE340E34DF34CF3473
:1032A000E1348D34E3344634E434F934E634A6347E
:1032B000E8344C34E934EA34EB347F34ED340A3406
:1032C000EE348B34F0340134F1346B34F234C934DD
:1032D000F4341934F5345B34F6348E34F734B234C4
:1032E000F834C634F934C934FA34BB34FB349A3474
:1032F000FC346734FD342134FD34C734FE34583493
:10330000FE34D534FF343D34FF348F34FF34CB34B6
:10331000FF34F134FF34FF34FF34F734FF34D63454
:10332000FF349E34FF344E34FE34E634FE346534CC
:10333000FD34CC34FD341934FC344E34FB346A345F
:10334000FA346D34F9345634F8342734F634DF3433
:10335000F5347D34F4340334F2347134F034C6344B
:10336000EF340234ED342734EB343434E9342A3486
:10337000E7340834E434D034E2348134E0341C34AB
:10338000DD34A234DB341234D8346E34D534B63460
:10339000D234EB34D0340D34CD341C34CA34193427
:1033A000C7340634C334E234C034AE34BD346C3474
:1033B000BA341B34B634BC34B3345134AF34DA3499
:1033C000AC345734A834CB34A5343434A1349534D8
:1033D0009D34EE349A34403496348B349234D23463
:1033E0008F3413348B34523487348D348334C73460
:1033F000803400347C343934783473347434AE34EB
:103400007034ED346D342E34693475346534C03421
:10341000623412345E346B345A34CC34573435341D
:103420005334A934503426344C34AF344934443402
:103430004534E534423494343F3452343C341E3401
:103440003834FA343534E7343234E4342F34F33456
:103450002D3415342A344A34273492342434EE344B
:1034600022345E341F34E4341D347F341B34303452
:103470001834F8341634D6341434CC341234D934E5
:103480001034FE340F343A340D348F340B34FD34A1
:103490000A348334093421340734D9340634AA3445
:1034A00005349334043496340334B2340234E734AC
:1034B0000234343401349B3401341A340034B234CD
:1034C0000034623400342A340034093400340134C6
:1034D00000340F3400343534003471340034C334D4
:1034E00001342B340134A834023439340234DF344B
:1034F000033499340434663405344534063437349F
:1035000007343A3408344E34093472340A34A5345A
:103510000B34E7340D3437340E3495340F34FF3424
:10352000113475341234F6341434813416341634AC
:103530001734B43419345A341B3407341C34BA34B5
:103540001E347334203431342134F2342334B7340C
:1035500025347E3427344734293410342A34D9347E
:103560002C34A1342E34683430342C343134EC34DF
:103570003334A93435346134373413343834BF34F8
:103580003A3463343C3400343D3495343F34203491
:103590004034A23442341934433485344434E5345D
:1035A00046343934473480344834BA344934E53405
:1035B0004B3403344C3411344D3411344E34003414
:1035C0004E34E0344F34AE3450346C34513419340A
:1035D0005134B53452343E345234B63453341C343E
:1035E000533470345334B1345334DF345334FB34F4
:1035F000543404345334FB345334DF345334B1344F
:103600005334703453341C345234B63452343E3450
:103610005134B5345134193450346C344F34AE34E1
:103620004E34E0344E3400344D3411344C341134C3
:103630004B3403344934E5344834BA3447348034A5
:10364000463439344434E53443348534423419340F
:103650004034A2343F3420343D3495343C3400347B
:103660003A3463343834BF34373413343534613446
:103670003334A9343134EC3430342C342E346834BF
:103680002C34A1342A34D934293410342734473423
:1036900025347E342334B7342134F23420343134A9
:1036A0001E3473341C34BA341B34073419345A347E
:1036B0001734B43416341634143481341234F634D6
:1036C000113475340F34FF340E3495340D343734DF
:1036D0000B34E7340A34A5340934723408344E34D8
:1036E00007343A3406343734053445340434663408
:1036F000033499340234DF34023439340134A834C9
:1037000001342B340034C334003471340034353484
:1037100000340F34003401340034093400342A34C6
:10372000003462340034B23401341A3401349B342E
:10373000023434340234E7340334B234043496347B
:10374000053493340634AA340734D9340934213487
:103750000A3483340B34FD340D348F340F343A344F
:103760001034FE341234D9341434CC341634D634F4
:103770001834F8341B3430341D347F341F34E434AF
:1037800022345E342434EE34273492342A344A34DA
:103790002D3415342F34F3343234E4343534E734F3
:1037A0003834FA343C341E343F3452344234943486
:1037B0004534E534493444344C34AF345034263441
:1037C0005334A934573435345A34CC345E346B34E2
:1037D000623412346534C034693475346D342E3437
:1037E0007034ED347434AE34783473347C3439341A
:1037F00080340034803400348334A9348734513425
:103800008A34F5348E34943492342C349534BC3468
:10381000993442349C34BC34A0342934A3348734E2
:10382000A634D534AA341134AD343934B0344D34DF
:10383000B3344B34B6343234B9340034BB34B434DA
:10384000BE344D34C034CB34C3342B34C5346E3421
:10385000C7349234C9349634CB347B34CD343E34BF
:10386000CE34E034D0346034D134BE34D234F93480
:10387000D4341234D5340734D534DA34D6348934D8
:10388000D7341534D7347F34D734C634D734EB34F7
:10389000D734EE34D734D034D7349134D7343134AC
:1038A000D634B334D6341634D5345B34D43483347C
:1038B000D3349034D2348134D1345934D03419349F
:1038C000CE34C134CD345334CB34D134CA343B3408
:1038D000C8349434C634DC34C5341534C33441346C
:1038E000C1346134BF347734BD348434BB348B3459
:1038F000B9348B34B7348834B5348334B3347E343C
:10390000B1347934AF347734AD347A34AB34823473
:10391000A9349234A734AC34A534D034A434003460
:10392000A2343D34A0348A349E34E7349D34553477
:103930009B34D7349A346D34993419349734DB344A
:103940009634B5349534A7349434B3349334D9349D
:1039500093341B34923479349134F33491348B346E
:103960009134403491341434913406349134163403
:1039700091344634913495349234033492349034F3
:1039800093343C34943407349434F0349534F7341D
:1039900097341B3498345D349934BB349B343534BC
:1039A0009C34CA349E347934A0344134A234223455
:1039B000A4341934A6342734A8344A34AA348134C0
:1039C000AC34CA34AF342534B1348F34B434083411
:1039D000B6348D34B9341E34BB34BA34BE345D349D
:1039E000C1340834C334B734C6346A34C9342034DB
:1039F000CB34D534CE348934D1343A34D334E6346C
:103A0000D6348C34D9342A34DB34BF34DE344834F1
:103A1000E034C434E3343234E5349034E734DC3415
:103A2000EA341534EC343A34EE344934F034413469
:103A3000F2342134F334E634F5349134F7341F345E
:103A4000F8349134F934E434FB341834FC342C3435
:103A5000FD342034FD34F234FE34A134FF342E34EE
:103A6000FF349734FF34DD34FF34FE34FF34FC344C
:103A7000FF34D434FF348834FF341734FE348234B6
:103A8000FD34C834FC34EA34FB34E834FA34C2344C
:103A9000F9347934F8340D34F6348034F434D134D4
:103AA000F3340134F1341234EF340434EC34D934C7
:103AB000EA349034E8342C34E534AE34E33416344C
:103AC000E0346634DD349F34DA34C434D734D4344B
:103AD000D434D234D134BF34CE349D34CB346D346D
:103AE000C8343134C434EA34C1349B34BE34443431
:103AF000BA34E834B7348834B4342634B034C434F7
:103B0000AD346234AA340434A634AA34A33457340E
:103B1000A0340B349C34C9349934923496346734CD
:103B200093344B3490343E348D3442348A34583498
:103B3000873483348434C234823418347F348534F7
:103B40007D340B347A34AA347834643476343A349D
:103B500074342C3472343B34703468346E34B4347E
:103B60006D341F346B34A9346A34533469341E34D1
:103B700068340934673414346634413465348E341F
:103B80006434FC3464348A3464343934643407343F
:103B90006334F5346434023464342D34643477345B
:103BA0006434DD3465345F346534FD346634B634F2
:103BB0006734883468347334693475346A348D34C6
:103BC0006B34BA346C34FB346E344F346F34B334EA
:103BD000713427347234A934743438347534D2349F
:103BE00077347534793421347A34D3347C348A345C
:103BF0007E344434803400348134BC3483347634AD
:103C000085342D348634DF3488348B348A342E3432
:103C10008B34C8348D3457348E34D93490344D3489
:103C20009134B13493340534943446349534733438
:103C300096348B3497348D349834783499344A34AC
:103C40009A3403349A34A1349B3423349B3489341A
:103C50009B34D3349B34FE349C340B349B34F93482
:103C60009B34C7349B3476349B3404349A34723496
:103C70009934BF349834EC349734F7349634E234C2
:103C80009534AD34943457349234E13491344C3417
:103C90008F3498348D34C5348B34D4348934C6345D
:103CA00087349C34853456348234F53480347B3404
:103CB0007D34E8347B343E3478347D347534A83434
:103CC0007234BE346F34C2346C34B53469349934D0
:103CD00066346E34633437345F34F5345C34A9347D
:103CE000593456345534FC3452349E344F343C34B9
:103CF0004B34DA3448347834453418344134BC34E5
:103D00003E3465343B3416343734CF343434933452
:103D1000313463342E3441342B342E3428342C3453
:103D200025343C34223461341F349A341C34EA3450
:103D30001A3452341734D4341534703413342734CD
:103D40001034FC340E34EE340C34FF340B342F3486
:103D5000093480340734F3340634873405343E3470
:103D600004341834033416340234383401347E34C5
:103D70000034E9340034783400342C340034043412
:103D80000034023400342334003469340034D23433
:103D900001345F3402340E340234E0340334D4345A
:103DA0000434E83406341C3407346F340834E13406
:103DB0000A346F340C341A340D34DF340F34BF340A
:103DC0001134B7341334C6341534EB341834243476
:103DD0001A3470341C34CE341F343C342134B8349B
:103DE000243441342634D634293474342C341A34EF
:103DF0002E34C6343134773434342B343634E03412
:103E0000393496343C3449343E34F8344134A334A4
:103E1000443446344634E234493473344B34F83451
:103E20004E3471345034DB345334363455347F34AB
:103E30005734B6345934D9345B34E7345D34DE3426
:103E40005F34BF3461348734633436346434CB3404
:103E5000663445346734A3346834E5346A3409344D
:103E60006B3410346B34F9346C34C4346D347034C6
:103E70006D34FD346E346B346E34BA346E34EA34DF
:103E80006E34FA346E34EC346E34C0346E347534BF
:103E90006E340D346D3487346C34E5346C3427342F
:103EA0006B344D346A34593469344B3468342534B6
:103EB0006634E73465349334643429346234AB3483
:103EC000613419345F3476345D34C3345C34003487
:103ED0005A3430345834543456346E3454347E3476
:103EE00052348634503489344E3487344C348234DE
:103EF0004A347D3448347834463475344434753427
:103F000042347C34403489343E349F343C34BF34B2
:103F10003A34EB343934243437346C343534C534E2
:103F200034342F343234AD3431343F342F34E73429
:103F30002E34A7342D347F342C3470342B347D341C
:103F40002A34A5342934EA3429344D342834CF3482
:103F500028346F342834303428341234283415345B
:103F600028343A34283481342834EB3429347734F3
:103F70002A3426342A34F9342B34EE342D340734E1
:103F80002E3442342F34A034313420343234C2340D
:103F90003434853436346A3438346E343A349234B6
:103FA0003C34D5343F3435344134B33444344C3468
:103FB000473400344934CE344C34B5344F34B33400
:103FC0005234C7345534EF3459342B345C3479349B
:103FD0005F34D734633444346634BE346A34443492
:103FE0006D34D43471346C3475340B347834AF346C
:083FF0007C34573480340034A6
:043FF800003400345D
:020000040001F9
:02000E00840963
:02001000FF1FD0
:00000001FF
